:020000040000FA
:10000000831600308600850083123830502001307E
:100010005020033050200F30502080305020831665
:10002000F030860081138312EF309F008600043089
:10003000A0009F0C1F088600682006080F38A1004A
:10004000A109031D2628A00B1928142806080F381B
:10005000A400A409031D26288316003086008312FD
:100060009F091F080F399F002108F0399F041F08BE
:1000700086001130A100A103210870201F02031D7A
:100080003B282108860010302107702086009F0041
:10009000003083160030860083121F085C200F2872
:1000A00086006820043085006820003085006820C4
:1000B000043085006820080086006820063085002E
:1000C000682002308500682006308500682008001E
:1000D0003230A300A200A20B6B28A30B6A280800F1
:1000E0008207113412341434183421342234243465
:1000F00028344134423444344834813482348434A2
:100100008834303431343234333434343534363462
:100110003734383439344134423443344434453448
:02012000463463
:02400E00F13F80
:00000001FF
